:100000000C947B000C94A3000C94A3000C94610549
:100010000C9461050C9461050C94A3000C94A3004E
:100020000C94A3000C94A3000C94A3000C94A300C4
:100030000C94A3000C94A3000C94A3000C94A300B4
:100040000C9417050C94A3000C94A3000C94A3002B
:100050000C94A3000C94A3000C94A3000C94A30094
:100060000C94A3000C94A3000000000024002700BF
:100070002A0000000008000201000003040700003D
:1000800000000000000000000000230026002900FE
:1000900000000000250028002B00040404040404D0
:1000A0000404020202020202030303030303010227
:1000B00004081020408001020408102001020408F6
:1000C00010205600566F6C7461676500566F6C7433
:1000D0000020566F6C7453656E736F7220312E3230
:1000E0000020534542492050696C6F742020202025
:1000F0000000F3050E0811241FBECFEFD8E0DEBFCD
:10010000CDBF11E0A0E0B1E0ECEEF3E102C005905C
:100110000D92A231B107D9F722E0A2E1B1E001C00E
:100120001D92AD30B207E1F710E0CAE7D0E004C09D
:100130002197FE010E94E309C937D107C9F70E9440
:1001400027060C94E9090C9400000895AF92BF9221
:10015000CF92DF92EF92FF920F931F93CF93DF9393
:100160006C017B018B01040F151FEB015E01AE18C2
:10017000BF08C017D10759F06991D601ED91FC91E4
:100180000190F081E02DC6010995892B79F7C50111
:10019000DF91CF911F910F91FF90EF90DF90CF9063
:1001A000BF90AF90089590E0FC01EE58FF4F24916E
:1001B000FC01E255FF4F3491FC01E656FF4FE491FC
:1001C000EE23C9F0222339F0233001F1A8F42130C5
:1001D00019F1223029F1F0E0EE0FFF1FE057FF4F39
:1001E000A591B4918FB7F894EC91611126C0309528
:1001F0003E233C938FBF08952730A9F02830C9F0E3
:10020000243049F7809180008F7D03C08091800069
:100210008F7780938000DFCF84B58F7784BDDBCF6D
:1002200084B58F7DFBCF8091B0008F778093B00035
:10023000D2CF8091B0008F7DF9CF3E2BDACFCF9314
:10024000DF9390E0FC01E255FF4F249186569F4FCB
:10025000FC0184918823C9F090E0880F991FFC016C
:10026000E859FF4FA591B491FC01E057FF4FC591AC
:10027000D49161110DC09FB7F8948C912095822381
:100280008C938881282328839FBFDF91CF91089585
:10029000623051F49FB7F8943C91822F809583236C
:1002A0008C93E8812E2BEFCF8FB7F894EC912E2B07
:1002B0002C938FBFEACF862798E027E087FF05C001
:1002C000880F82279150D1F70895880FFBCFDC016A
:1002D0005196ED91FC915297908150968C9180951A
:1002E00089238083089520913301309134012817A8
:1002F000390771F49091310180913201981741F0E2
:10030000E0913101F0E0EC5EFE4F808190E00895D5
:100310008FEF9FEF089508952091330130913401BC
:100320002817390769F4809132012091310190E05A
:100330004096821B910960E170E00E94BB0908951C
:1003400090E080E008952091330130913401281726
:100350003907B9F49091310180913201981789F0F1
:10036000E0913101F0E0EC5EFE4F8081209131019F
:1003700030E02F5F3F4F2F7033272093310190E003
:1003800008958FEF9FEF0895E0913301F0913401CC
:10039000E817F90769F4A389B4899C918589809548
:1003A00089238C93109234011092330181E00895D7
:1003B00080E00895CF93DF938AE391E00E94C40127
:1003C000CAE3D1E061E08C850E941F0161E08C8569
:1003D000DF91CF910C94D3008091570190915801F7
:1003E000892B31F1809133019091340121E08A33DE
:1003F0009207F1F0009711F00E94C4018091510121
:100400008E7F8093510110923201109231018AE364
:1004100091E09093340180933301E0914D01F0918C
:100420004E01808190914F01892B808381E0089556
:1004300080E0089590E080E00895CF92DF92EF92FF
:10044000FF920F931F93CF93DF93EC0189A19AA1A1
:10045000892B79F481E090E09B838A8390E080E0AF
:10046000DF91CF911F910F91FF90EF90DF90CF9090
:1004700008950FB7F8948F8D98A110E0892B89F01B
:1004800028E030E080E091E0462F492309F08F5FBB
:10049000990F21503109C1F7988D91118F5F182F55
:1004A0001095F62ECE010E94670189A19AA10197AD
:1004B000F1F788E0C82ED12CEE24E3948F2D8E2105
:1004C00009F43DC0E989FA8980819889892B808364
:1004D00089A19AA10197F1F7EE0C81E0C81AD10821
:1004E00069F78E89882369F0888D882361F1E9890D
:1004F000FA8980819889892B808389A19AA10197A3
:10050000F1F78F8D98A1892B61F010FF20C0E98948
:10051000FA8980819889892B80838F8D98A1019792
:10052000F1F7E989FA8980819889892B80830FBF47
:100530008D8D9E8D0197F1F781E090E091CFCE01F6
:100540000E946701C5CFCE010E946701D6CFCE01C0
:100550000E946701E2CF2F923F924F925F926F927B
:100560007F928F929F92AF92BF92CF92DF92EF9243
:10057000FF920F931F93CF93DF9380900702909089
:100580000802A0900902B0900A0224EF820E21E036
:10059000921EA11CB11C8FB7F89440903501509069
:1005A000360160903701709038018FBF1092520170
:1005B0006EE78AE391E00E941D02D1E0D0935201E0
:1005C0006FE98AE391E00E941D0284149504A60459
:1005D000B70408F424C18091E001E0915D01F0913D
:1005E0005E01A82FB0E0AA0FBB1FA154BE4F2D91F2
:1005F0003C91232B09F409C18093E0016091E00153
:10060000A6E0C6E0D0E050E040E010E070E09A01E3
:10061000260F371F2E173F07D4F42115310569F037
:100620001F5F220F331FD901A156BE4F2C912F718E
:10063000DE01283009F4F1C021964F5F5F4F403151
:10064000510529F0CB31D10514F31150CA2FC064E4
:1006500081E0809352016C2F8AE391E00E941D0299
:1006600060E08C2F0E945B01C82FDD24D394D092D0
:10067000520161E18AE391E00E941D026C2F81E149
:100680000E945B01C82FD092520164EA8AE391E094
:100690000E941D026C2F84EA0E945B01C82FD09239
:1006A000520169E58AE391E00E941D026C2F89E501
:1006B0000E945B01C82FD092520169E08AE391E069
:1006C0000E941D026C2F89E00E945B01C82FD0920E
:1006D000520160E08AE391E00E941D0210925201F3
:1006E0006C2F80E00E945B01D82F84149504A6042F
:1006F000B70408F4FCC0C091E0011C0F01E0809138
:100700005D0190915E011C1709F4A6C077247394D3
:100710007C0E7092E001CC2ED12CC816D9060CF0BC
:100720009BC0CC2309F46FC0E0910B02F0910C0246
:100730000995C601880F991FFC01E156FE4F7F0104
:1007400080818F71883009F05EC0C295C07FC8601B
:10075000009352016C2F8AE391E00E941D026D2FDD
:100760008C2F0E945B01C82FF601EE0FFF1FE15492
:10077000FE4F0190F081E02D80809180A280B380B7
:10078000FFE9BF2200935201682D8AE391E00E94A5
:100790001D026C2F882D0E945B01C82F292C3A2C3A
:1007A0004B2C552447FC5A9400935201622D8AE346
:1007B00091E00E941D026C2F822D0E945B01C82FC8
:1007C0001501552437FC5094452C00935201622D9D
:1007D0008AE391E00E941D026C2F822D0E945B0132
:1007E000D82FF701C081C07ECB29009352016C2F16
:1007F0008AE391E00E941D02109252016D2F8C2F0E
:100800000E945B01D82FC72D7ACF8F5F8E171F06EE
:100810000CF4E7CE1092E001F1CE25960ECFE091D8
:100820003901F0E0EE0FFF1FE056FE4F8081C82F28
:10083000CF71829586958770C80FC85FD09352019B
:100840006C2F8AE391E00E941D0260E08C2F0E94D1
:100850005B01C82F10E009CF2091E0010197281714
:10086000190614F01092E00181E0809352016D2F7F
:100870008AE391E00E941D0210925201E0910B0266
:10088000F0910C020995109252016EEF8AE391E00B
:100890000E941D02C5EED1E005E012E0FF24F394B2
:1008A0006991F09252018AE391E00E941D02109238
:1008B00052010C171D07A1F76FEF8AE391E00E9428
:1008C0001D021092520181E0DF91CF911F910F9193
:1008D000FF90EF90DF90CF90BF90AF909F908F9060
:1008E0007F906F905F904F903F902F900895C091B0
:1008F0003901D09252016C2F8AE391E00E941D02CF
:100900006D2F8C2F0E945B01D82F0C2F10E07801E7
:10091000EE0CFF1C970120563E4F5901F9018081D2
:10092000982F9F71F8E09F9F400111248295869532
:100930008770882AD0925201682D8AE391E00E9444
:100940001D02109252016D2F882D0E945B01D82F3D
:10095000F701E15AFE4F80809180D12CC12C662492
:100960006394F50180818F71C816B0F4F401EC0D29
:10097000FD1D749060925201672D8AE391E00E9400
:100980001D02109252016D2F872D0E945B01D82FFE
:10099000FFEFCF1ADF0AE5CF000F111FF801E15872
:1009A000FE4FC080D18010E000E0970120563E4FFE
:1009B0005901EE24E394F501808182958695877034
:1009C0000817A8F4F601E00FF11FF490E09252012D
:1009D0006F2D8AE391E00E941D02109252016D2F4B
:1009E0008F2D0E945B01D82F0F5F1F4FE4CFCF5F89
:1009F000C093390180915D0190915E01C81719067D
:100A000014F0109239012FB7F8948091350190912C
:100A10003601A0913701B09138012FBF80930702B2
:100A200090930802A0930902B0930A021DCF1F926F
:100A30000F920FB60F9211242F933F938F939F9392
:100A4000AF93BF938091350190913601A09137010A
:100A5000B09138013091280123E0230F2D3758F54C
:100A60000196A11DB11D209328018093350190931B
:100A70003601A0933701B093380180912401909101
:100A80002501A0912601B09127010196A11DB11D5C
:100A90008093240190932501A0932601B093270110
:100AA000BF91AF919F918F913F912F910F900FBE6A
:100AB0000F901F90189526E8230F0296A11DB11DD7
:100AC000D2CF1F920F920FB60F9211242F933F9304
:100AD0004F935F936F937F938F939F93AF93BF9346
:100AE000CF93DF93EF93FF93E0913301F0913401C3
:100AF000309709F45DC0C685D785888155858523E3
:100B000009F056C0818D928D0197F1F7238D348DB8
:100B100068E070E040E081E0D9011197F1F7988139
:100B2000952309F458C0482B880F61507109A1F72B
:100B30008091320190E001968F7099276091310188
:100B4000681709F44CC0A0913201B0E0AC5EBE4F12
:100B50004C938093320186898823D1F0C901019793
:100B6000F1F72881252381E090E0A0E0B0E004C007
:100B7000880F991FAA1FBB1F2A95D2F72091120137
:100B800030911301822B932B9093130180931201C8
:100B9000878D90A1009711F00197F1F7858D968DC3
:100BA0000197F1F7A389B4898C919589892B8C934E
:100BB000FF91EF91DF91CF91BF91AF919F918F9175
:100BC0007F916F915F914F913F912F910F900FBE49
:100BD0000F901F901895982F90954923A5CF87893E
:100BE0008160878BB8CFEAE3F1E01382128288EE4E
:100BF00093E0A0E0B0E084839583A683B78384E08C
:100C000091E091838083A1E5B1E08C918E7F8C93FC
:100C1000128E118E148E138E168E158E12A211A2A4
:100C20001092E1011092E2011092E3011092E401AE
:100C30001092DF0110925E0110925D011092E001AE
:100C400085EA90E090930C0280930B0208957894CB
:100C500084B5826084BD84B5816084BD85B58260C1
:100C600085BD85B5816085BD80916E008160809372
:100C70006E001092810080918100826080938100DB
:100C800080918100816080938100809180008160EB
:100C9000809380008091B10084608093B100809146
:100CA000B00081608093B00080917A00846080936E
:100CB0007A0080917A00826080937A0080917A0035
:100CC000816080937A0080917A00806880937A00B6
:100CD0001092C10061E08DE00E941F0161E08DE093
:100CE0000E94D30061E083E00E941F0160E083E086
:100CF0000E94D300A5EEB1E0E1EEF0E080E090E2EA
:100D00008F3009F485C19F012F5F3F4FE491EC9331
:100D1000F9018F5F1196803199F7A5EFB1E0E1ED10
:100D2000F0E080E090E28F3009F475C19F012F5F01
:100D30003F4FE491EC93F9018F5F1196803199F761
:100D40008CEC90E09093600180935F0110928001A1
:100D500010927F011092C0011092BF0110929F016A
:100D600084E08093A00181E090E090935E01809305
:100D70005D0161E083E00E94D30061E083E00E94B6
:100D80001F0101EB10E0F801849180934A01CDE945
:100D9000D0E0FE018491E82FF0E0EE0FFF1FE05756
:100DA000FF4F8591949190934C0180934B0160E0AB
:100DB00083E00E941F0161E083E00E94D30083E092
:100DC00080934601F801049100934701FE01C4910C
:100DD000EC2FF0E0EE0FFF1FEA57FF4F8591949143
:100DE000909349018093480181E08093500185E907
:100DF00091E090935C0180935B0129EB30E03093AC
:100E000054012093530123E931E03093560120939C
:100E1000550146E554E050935801409357013093F3
:100E20005A012093590120916800246020936800A2
:100E30002DE630E030934E0120934D0128E02093C1
:100E40004F010197F1F70E94EC010E94DA0162E084
:100E500085E00E941F018EED97EAA8E3BEE3809330
:100E60002D0190932E01A0932F01B093300120917A
:100E70005D0130915E01203131050CF040C0C901A7
:100E80000196FC01EE0FFF1FE35AFE4F44EC50E0C9
:100E900051834083F901EE0FFF1FE158FE4F42ECF2
:100EA00050E051834083F901EE0FFF1FE154FE4FE4
:100EB00011821082F901EE0FFF1FE156FE4F1082E2
:100EC000220F331FF901E056FE4F27E22083909353
:100ED0005E0180935D018150803188F490E0FC01D7
:100EE000EE0FFF1FE154FE4F29E231E031832083F2
:100EF000880F991FFC01E156FE4F88E480830E9411
:100F0000AB0260E08DE00E94D30012E4C0E0D0E0CC
:100F100010937C0080917A00806480937A008091A5
:100F20007A0086FDFCCF8091780060917900762F61
:100F3000682F072E000C880B990B0E94C20820E036
:100F400030EC4FE754E40E94180820E030E040EA1B
:100F500050E40E944E0920912D0130912E014091C4
:100F60002F01509130010E94180820E030E048EC39
:100F700052E40E944E090E948A08609329017093EE
:100F80002A0180932B0190932C0161E08DE00E9457
:100F9000D3008AE391E00E94C4010E94DA010E941A
:100FA000AB0260E0809146010E941F0161E08091E8
:100FB00046010E94D3000E94EC010E94EC0160E017
:100FC0008DE00E94D3002FB7F89480913501909165
:100FD0003601A0913701B09138012FBF8C599F4F36
:100FE000AF4FBF4F2FB7F894409135015091360164
:100FF00060913701709138012FBF481759076A0770
:101000007B0780F3209709F483CF0E94000080CFF4
:101010009093F4017ECE909304028ECE84E091E012
:1010200090933B0180933A018AE391E00C94C401D0
:101030000E942C080C9414090E940D0958F00E947B
:10104000060940F029F45F3F29F00C94FD08511186
:101050000C9448090C9403090E94250968F399230C
:10106000B1F3552391F3951B550BBB27AA276217A4
:101070007307840738F09F5F5F4F220F331F441FB1
:10108000AA1FA9F335D00E2E3AF0E0E832D09150E5
:101090005040E695001CCAF72BD0FE2F29D0660FD2
:1010A000771F881FBB1F261737074807AB07B0E815
:1010B00009F0BB0B802DBF01FF2793585F4F3AF01B
:1010C0009E3F510578F00C94FD080C9448095F3F51
:1010D000E4F3983ED4F3869577956795B795F795A1
:1010E0009F5FC9F7880F911D9695879597F9089589
:1010F000E1E0660F771F881FBB1F62177307840725
:10110000BA0720F0621B730B840BBA0BEE1F88F733
:10111000E09508950E9491086894B1110C944809D3
:1011200008950E942D0988F09F5798F0B92F9927AC
:10113000B751B0F0E1F0660F771F881F991F1AF0C2
:10114000BA95C9F714C0B13091F00E944709B1E0D7
:1011500008950C944709672F782F8827B85F39F0D6
:10116000B93FCCF3869577956795B395D9F73EF45B
:1011700090958095709561957F4F8F4F9F4F089503
:10118000E89409C097FB3EF4909580957095619521
:101190007F4F8F4F9F4F9923A9F0F92F96E9BB27D7
:1011A0009395F695879577956795B795F111F8CF53
:1011B000FAF4BB0F11F460FF1BC06F5F7F4F8F4FBE
:1011C0009F4F16C0882311F096E911C0772321F0B4
:1011D0009EE8872F762F05C0662371F096E8862F4C
:1011E00070E060E02AF09A95660F771F881FDAF7A3
:1011F000880F9695879597F9089597F99F6780E8E6
:1012000070E060E008959FEF80EC089500240A9458
:101210001616170618060906089500240A941216D1
:101220001306140605060895092E0394000C11F404
:10123000882352F0BB0F40F4BF2B11F460FF04C0B1
:101240006F5F7F4F8F4F9F4F089557FD9058440F0A
:10125000551F59F05F3F71F04795880F97FB991F15
:1012600061F09F3F79F087950895121613061406D2
:10127000551FF2CF4695F1DF08C01616170618065F
:10128000991FF1CF86957105610508940895E8943A
:10129000BB2766277727CB0197F908950E9461093C
:1012A0000C9414090E94060938F00E940D0920F0E0
:1012B000952311F00C94FD080C94030911240C944F
:1012C00048090E94250970F3959FC1F3950F50E0DE
:1012D000551F629FF001729FBB27F00DB11D639FE8
:1012E000AA27F00DB11DAA1F649F6627B00DA11D8E
:1012F000661F829F2227B00DA11D621F739FB00D34
:10130000A11D621F839FA00D611D221F749F3327A3
:10131000A00D611D231F849F600D211D822F762F3C
:101320006A2F11249F5750409AF0F1F088234AF019
:10133000EE0FFF1FBB1F661F771F881F9150504085
:10134000A9F79E3F510580F00C94FD080C944809C4
:101350005F3FE4F3983ED4F3869577956795B7950C
:10136000F795E7959F5FC1F7FE2B880F911D969526
:10137000879597F9089597FB072E16F4009407D0E8
:1013800077FD09D00E94CF0907FC05D03EF4909567
:1013900081959F4F0895709561957F4F0895AA1B81
:1013A000BB1B51E107C0AA1FBB1FA617B70710F050
:1013B000A61BB70B881F991F5A95A9F78095909582
:1013C000BC01CD010895EE0FFF1F0590F491E02DB3
:1013D000099410E0CAE7D0E004C0FE010E94E309CE
:0C13E0002196CB37D107C9F7F894FFCF56
:1013EC00000000001D02A6001A028B018C01A30153
:0213FC0073017B
:00000001FF
